:020000040000FA
:02000000ED28E9
:08000800A200030EA1000B1E73
:100010000B288B180E280B19142842283C30A800F6
:1000200067200B128B1042284720A003031D1A28BB
:100030000430A00001302002031D23281C3085005D
:100040002608A7003E2802302002031D2C281A3063
:1000500085002508A7003E2803302002031D35280F
:10006000163085002408A7003E2804302002031D16
:100070003E280E3085002308A7003E289D204F20F3
:100080000B114228210E8300A20E220E09000B1A2A
:100090000800A803031D08000B168B100800861C1F
:1000A00054282C1854282A142C1086182C142B1C75
:1000B0006028A90303195D2808002B102A100800E6
:1000C0002A1C08002B143C30A90080200800A30A39
:1000D0000A302302031D0800A301A40A0A302402E7
:1000E000031D0800A401A50A0A302502031D08000B
:1000F000A501A60A0A302602031D0800A601080071
:10010000A303FF302302031D08000930A300A4034A
:10011000FF302402031D08000930A400A503FF30AE
:100120002502031D08000930A500A603FF302602A2
:10013000031D08000930A600080000302702031D37
:10014000A528003086000514080001302702031D91
:10015000AD28E43086000514080002302702031D94
:10016000B528903086000510080003302702031DD3
:10017000BD28C03086000510080004302702031D8A
:10018000C528643086000510080005302702031DCD
:10019000CD28483086000510080006302702031DD0
:1001A000D5280C3086000510080007302702031DF3
:1001B000DD28E03086000514080008302702031D02
:1001C000E528003086000510080009302702031DCD
:1001D00008006030860005100800831203138501B3
:1001E000860107309F0083160313453081000030DD
:1001F00085000330860083120313B0308B00850125
:100200008101A601A501A401A301A7010430A0005A
:100210003C30A800A900AA01AB012C140F290F291A
:02400E00223F4F
:00000001FF
